:020000040800F2
:100000000002002029050008C5040008810400083A
:10001000D5040008E5040008F5040008000000000D
:10002000000000000000000000000000450400087F
:100030000505000800000000290400081505000857
:100040008901000889010008890100088901000868
:1000500089010008890100086D1600086D16000866
:100060006D1600086D1600086D160008890100085D
:100070008901000889010008890100088901000838
:100080008901000889010008890100088901000828
:100090008901000889010008890100086D1600081F
:1000A0008901000889010008890100088901000808
:1000B0000518000889010008890100088901000865
:1000C00089010008890100088901000889010008E8
:1000D00089010008890100081D1200082312000888
:1000E0006D160008890100088901000889010008CF
:1000F00089010008890100088901000889010008B8
:1001000089010008890100080B180008890100080E
:100110008901000889010008890100088901000897
:100120008901000889010008890100088901000887
:100130008901000889010008890100088901000877
:100140008901000889010008890100088901000867
:100150008901000889010008890100088901000857
:100160008901000889010008890100088901000847
:1001700089010008890100088901000800000000C9
:10018000000000008901000800F0C4B900F004BBC1
:100190007047000070B50C46064600F061F9094B47
:1001A000094A1D682919914202D8084A914204D28D
:1001B0000C2333604FF0FF3500E0196000F058F970
:1001C000284670BD000200200000022030120020EE
:1001D0001946104600F0ECBA1946104600F0F0BA85
:1001E000132303604FF0FF307047132303604FF079
:1001F000FF307047132303604FF0FF307047022930
:100200004FF0000303608CBF002001207047000006
:10021000114B70B500241C60104B114D18682E68EE
:1002200000F09CF80F4B53F820301B68A3F1080234
:1002300096420FD026B13179092904BF0A213171C4
:10024000092103F8041C33F9021C074B2A601980AA
:10025000012070BD204670BD94020020680300207C
:100260009C020020A402002098020020082930B53A
:10027000037919D9082B32D842791A4B53F82250F6
:1002800000F108042DB12D68856053F822502C60D0
:1002900000E0846043F82240134C4279012303FAC2
:1002A00002F22368134319E0082B18D945790D4B46
:1002B00053F825203AB11468A2420BBF00222468EB
:1002C00043F825201460427953F822303BB9064C9C
:1002D000012303FA02F2236823EA02032360017177
:1002E00030BD00BFA40200206803002008B50A4BFF
:1002F0001B681A79082A02D95B7983420AD900F06F
:10030000BAF818B1054B01221A6008BDBDE80840D3
:1003100000F082B808BD00BF9C02002094020020BB
:1003200008B500F09DF8094B094A1B88094D1BB21E
:10033000002442F82340084A286813682146013BFC
:100340001360FFF793FF2C6000F062F89802002022
:10035000E40200209C020020A00200200023C2072B
:1003600002D440080133FAE718467047134423F0DB
:10037000030310B54FF077321C1F43F8042C6207BB
:1003800042BF4FF0883243F8082CA3F108044FF025
:10039000807304E909000F4B44F80C3C002344F837
:1003A000103C032344F8143C2246022344F8183C32
:1003B000012344F81C3C42F8201D0B2342F8043D65
:1003C000013B032BFAD120466FF0020340F8443D75
:1003D00010BD00BF21030008064B0749074A1868F3
:1003E000884203D1934201D20433F8E70348C01A8C
:1003F000704700BF00000020FEE7FEE7000200207B
:10040000EFF30880704700000048704700000020AC
:1004100000F02AF801DFFEE7024A536843F08053F8
:100420005360704700ED00E0EFF3098020E9F00F22
:1004300040F804ED02490968086000F003F8000084
:100440009C020020FFF7E4FE04480068016801C92F
:10045000B1E8F00F81F30988004700009C020020FA
:10046000EFF3108072B6704762B6EFF310807047FA
:1004700080F310887047EFF30580C0B2704700002A
:100480000D490E4A0E4B6846904203D8984201D956
:10049000002102E009468D460121042072460242F5
:1004A00002D1EFF3088001E0EFF309802DE9F00FAE
:1004B0006B4600F06FF800BF000200200000022031
:1004C0006005002008B50249042000F079FB00BF58
:1004D000EC59000808B50249062000F071FB00BF86
:1004E000F859000808B50249072000F069FB00BF71
:1004F0000B5A000808B50249082000F061FB00BF54
:100500001D5A000808B50249092000F059FB00BF38
:10051000315A000808B502490A2000F051FB00BF1B
:10052000435A00087047704708B5FFF7FBFF6A465B
:10053000114B1249934202D243F8041BFAE7104AC6
:10054000104B11498B4204D252F8040F43F8040BAC
:10055000F8E70E4B0E4A0021934202D243F8041BE7
:10056000FAE7FFF7E0FF00F00BFB03F0DFFCBDE86C
:10057000084000F05DBB00BF00000020FEE7FEE782
:100580003866000800020020940200209402002037
:10059000301200202DE9F04F9A46494B8FB0934618
:1005A0009A6B03925A6B04929F6ADA6A05921A6BED
:1005B000DB6B0793434B06921A68434B9A420446FF
:1005C000884602D0414803F09BFFB8F1000F05D0E8
:1005D0003F48002503F094FF2E4626E094E80E00E5
:1005E000E068D4F81C9008902069099060690A902E
:1005F00019F4007F3748A6690D930CBF04F120055C
:1006000004F124050C920B9103F07AFF089B0093F0
:100610000BA90EC9304803F0E9FECDF8009033462F
:100620000A9A09992D4803F0E1FE2D4803F068FF6E
:1006300039462C4803F0DAFE05992B4803F0D6FE24
:1006400006992A4803F0D2FE0799294803F0CEFE06
:100650003A0403D50399274803F0C8FE3B0603D5A7
:100660000499254803F0C2FE244803F049FF594687
:10067000234803F0BBFEB8F1000F1BD1214803F063
:100680003FFF3146204803F0B1FE69461F4BC91AAF
:1006900003D549421E4803F0A9FE20468268C3687C
:1006A00001698C4641698E46AD46514691E8F00F8E
:1006B0004168006801BE1749052000F081FA00BFBB
:1006C00000ED00E000000020FEE7FEE7515A0008C0
:1006D000675A0008965A0008B15A0008EE5A0008F6
:1006E0002C5B0008355B0008455B0008555B000883
:1006F000655B0008755B0008855B0008955B00087A
:100700009A5B0008AC5B0008DD5B00085801002024
:10071000055C0008325C000810B568B1012815D1ED
:10072000174A136823F003031360136843F400733C
:1007300043F0010313601BE0114B1A6842F00E02F4
:100740001A605A6842F480725A6011E00D4A1369C7
:1007500023F0040313610024FFF782FEBFF34F8FE1
:1007600030BFFFF785FE54B1BDE8104000F0FABB82
:10077000044A136943F0040313610124ECE710BD3C
:100780000070004000ED00E008B5FFF769FE0020B2
:10079000BDE80840FFF7C0BF034B044A4FF4E13106
:1007A000002000F0B1BC00BF04020020FB0D0008D7
:1007B0000A460146014800F02BBB00BF040200209E
:1007C00010B50A460C460146002000F003FD204605
:1007D00010BD002000F0C0BF034B1968024611B9DC
:1007E000084600F099BF7047B003002010B5094AD1
:1007F00013685BB19C6881688C4202D21A461B6800
:10080000F7E703D15C6841688C42F7D90360106058
:1008100010BD00BFBC030020F0B51F4E1F4D336854
:100820001F4C013333601F4B00201A6818602B687F
:10083000226019460746B64641B1DEF800C08E6810
:10084000664503D80F4601200968F5E700B1296025
:1008500007B9F0BD00213960E2B133B15168586881
:10086000814294BF1146194600E0114608461268BD
:100870001B680AB903600BE00BB9026008E0556819
:100880005E68B54294BF15461D4605602846EEE7F2
:100890002160F0BD2360F0BDB4030020BC03002044
:1008A000B8030020AC0300202DE9F0412E4F2F4C5F
:1008B00001233B6023683BB9FFF7AEFFFFF789FFD9
:1008C0000130FBD0002502E0FFF783FF05464FF023
:1008D0000008236823B9FFF77CFF854214D91AE08A
:1008E0005E68FFF776FF854208D923685E68FFF7E8
:1008F00070FFA8422CD3B042F7D329E08642F4D946
:10090000361A132EE7D8F0E7236843B9FFF761FFE3
:10091000854206460BD9FFF77FFF0025D9E75E68C1
:10092000FFF757FF063E14308642D2D309E010F19C
:10093000140F04D3FFF74DFF8642FBD9EBE74FF0CE
:10094000FF3600233B603046BDE8F041FFF744BF6F
:1009500023681A682260C3F80480C3F80880DA6844
:1009600018699047B5E700BFB0030020B803002026
:10097000144B1A6882420AD112681A6012B1506888
:10098000063801E04FF0FF30FFF726BF13461A6824
:1009900022B19042FAD102681A6070470A4A13687D
:1009A0001BB1984203D01A46F9E7084A05E00368EC
:1009B000136070479842FAD01A461368002BF9D199
:1009C000704700BFB8030020AC030020BC03002028
:1009D00008B500231846054A054900F0CFFE4FF040
:1009E000FF30BDE80840FFF7F7BE00BFA9080008C8
:1009F00040420F00F8B504460D46FFF7EAFE00231B
:100A000085420646236010D3A5F10A0383420CD227
:100A10000A35FFF7DEFE8542FBD3FFF7DAFE85429B
:100A2000FBD8E368206998473EE0FFF719FD63684B
:100A30000746002B34D1A368002B31D11B4B6560D6
:100A40001A681B68B54238BF0132A260A2689A4298
:100A500003D92046FFF7CAFE1EE0B54202D9144B67
:100A600019460EE0134A136823B159688D4201D329
:100A70001A46F8E7236014600EE05068854203D3FD
:100A800013461A68002AF8D122601C600B689C4249
:100A900002D1A81FFFF7A0FE3846FFF7E9FC03E0EC
:100AA0002046FFF765FFC9E70020F8BDB40300202A
:100AB000B8030020AC03002038B50446FFF7D0FC93
:100AC0006368054633B9A36823B92846BDE83840B2
:100AD000FFF7CEBC2046FFF74BFFF6E7C36870B5C3
:100AE00004460D46C3B1FFF7E7FF092D0CD8FFF709
:100AF00070FE0646FFF76DFE801B8542FAD8E3685C
:100B00002069BDE870401847FFF763FE29182046AA
:100B1000BDE87040FFF76EBF70BD00002DE9F047E3
:100B200004460E4690461AB9BDE8F047FFF7D6BF17
:100B3000FFF796FC63680746E3B9A368D3B9DFF80B
:100B40003CA0FFF746FEDAF800508146FFF741FE71
:100B50008145F6D8304408EB0502864288BF013251
:100B60006060A2602046FFF741FE3846BDE8F047CE
:100B7000FFF77EBC2046FFF7FBFEE0E7B403002052
:100B800008B50121094800F099FC0121084800F04E
:100B900095FC0121074800F091FC0121064800F076
:100BA0008DFCBDE8084000F01FB900BF0D0C0240ED
:100BB0000C0C02400E0C02400F0C0240704700006B
:100BC00008B50F4B1A680C469AB9012203281A601F
:100BD00003D171460B4803F009FC21460A4803F093
:100BE00005FC00F04DF9094803F000FC084803F04B
:100BF000FDFBFFF735FCFFF7E1FFFFF7C5FD00BF89
:100C0000C0030020575C00085B5C0008835C0008A0
:100C1000775C000808B5034803F0E8FB00F058FED5
:100C2000002008BD855C000808B500F00BF9FCE762
:100C30001FB5FFF715FC0E4B0E481B6802930024EE
:100C40000D4B00930F220C234FF48071019400F0A0
:100C500055F80A4B0A481B6802930A4B0093072277
:100C60000C234FF4C061019400F048F8FFF7D0FB6B
:100C700018020020C4030020290C00081C020020D8
:100C8000C4040020150C000808B5FFF7E9FB094B68
:100C90001B681A79082A07D95A79074B53F822108A
:100CA00011B1096843F82210FFF7E2FBBDE80840E4
:100CB000FFF7B2BB9C020020A402002038B50B79DC
:100CC000082B03D908490320FFF77AFF4C7901F17B
:100CD000080203682BB113F8035CAC4201D3184639
:100CE000F7E78B60026038BD455C0008031F53F8CE
:100CF000042F9A42FBD0181A704700000F2A2DE9E2
:100D0000F74F05468B4691469A462AD810F00303C2
:100D10001BBFC3F10403ED180B46CB1A303B23F085
:100D200003031AF0080F05EB030405D02A46A2427C
:100D300003D212600432FAE72D600193FFF790FBB3
:100D40002749019B8046012251F8227016B25FB1FB
:100D50000132212AF8D14046FFF78AFB6FF08A0062
:100D60003BE06FF0150038E01D490C9841F8224037
:100D70002A46E6800D99FFF7F9FA0E9B194AA362FD
:100D80004FF0FF33E3611368206001331AF0010F65
:100D90006562C4F82CB084F805902771A760E760FD
:100DA00027616761A7612762136004D00121204693
:100DB000FFF75CFA0DE00A212046FFF757FA1AF018
:100DC000040F06D14046FFF753FB4846FFF78EFA63
:100DD00002E04046FFF74CFB304603B0BDE8F08F21
:100DE000E4020020A002002008B502F031F900F072
:100DF000B9F8BDE8084000F01CB838B50446043026
:100E000000F01BFD0546204601F0B8FF284638BD1E
:100E1000F8B504460E461746051D3A4631462846A3
:100E200000F0F6FC20B90121204601F077FFF4E73D
:100E3000F8BD08B5002000F01BFA0120BDE808400D
:100E400000F016BAF8B50D4B1E68C6F307221D4612
:100E500022B9F4B2003418BF012400E00224FFF7E5
:100E6000FFFA2B689E42074602D12046FFF754FC4A
:100E70003846BDE8F840FFF7FBBA00BF200200206B
:100E80002DE9F04F2C4B2D4A1B882D492D482E4E15
:100E9000DFF8CCB08BB00DF1280906F1800A29F8F3
:100EA000043D03F0A3FAFFF797FA0546FFF7ACFA03
:100EB0000446FFF7A5FA2A46009023464FF4007136
:100EC000224803F093FA25EAE5754FF4007856F8C6
:100ED000044B14B32779E26A5BF82730606A079302
:100EE00090440692FFF702FF069AB4F90610079B9A
:100EF000101A22680592626A04920390E26A0292D2
:100F000062790192082FD4BF4F4609F1010700977B
:100F10000544A26A0E4803F069FAB245D7D10D4BD9
:100F200002958DE808010C4A0C48194603F05EFA58
:100F30000BB0BDE8F08F00BFDD5C00080C5D000861
:100F4000125D0008175D0008E80200205F5D0008E0
:100F5000A95D0008E55D0008E75D0008EB5D00089D
:100F6000E05C000838B5FFF77BFA1B4C0023E36018
:100F7000054600F037F84FF41443A360A268164BFF
:100F800012F00C0FFAD1154A40F20571116081225E
:100F90001A601A6842F480321A601A6812F4003F2C
:100FA0000D4AFAD00E4B5360136843F08073136000
:100FB0001168094B8901FBD59A6842F002029A60D8
:100FC0009A6802F00C02082AFAD100F017F82846B5
:100FD000BDE83840FFF74CBA00380240003C024000
:100FE000042A4007044B1A6842F001021A601A688A
:100FF0009207FCD5704700BF00380240044B9A6846
:1010000012F00C0F1EBF1A6822F001021A6070471E
:1010100000380240034B044A00280CBF1046184613
:10102000704700BF00BD010580DE800204281CD887
:10103000DFE800F003080D1217000D4B1A6C114386
:10104000196412E00A4A536C194351640DE0084ACE
:10105000136B1943116308E0054A536B194351633D
:1010600003E0034A936B19439163BFF34F8F7047BB
:1010700000380240042821D8DFE800F003090F15EA
:101080001B000F4A136C23EA0101116470470C4ADC
:10109000536C23EA010151647047094A136B23EA38
:1010A000010111637047064A536B23EA0101516342
:1010B0007047034A936B23EA01019163704700BFB5
:1010C0000038024038B514230C4A4343D4582568ED
:1010D000AA0608D50A4B616803EBC002C9B253F8EF
:1010E0003030506898472B0748BF6368054B1B6832
:1010F0001BB1BDE83840FFF7C7BD38BD645E0008CE
:10110000C40A00209402002001282DE9F0478046FF
:101110000D46174603D92B490320FFF751FDDFF891
:10112000B090294A142404FB009442F83070E66819
:1011300002EBC00201215360304600F0BFF9304697
:1011400000F080FA3046617C00F054FA4E464FB110
:10115000D4F808900021484600F0B0F9217C4846B8
:1011600000F048FA142303FB08F806EB080999F885
:1011700012A0D9F804105046FFF758FF56F808405F
:101180000023E360504623616361FFF743FFB0FB38
:10119000F5F080B2A06077B199F8133001215AB20E
:1011A00003F01F0301FA03F35209084941F8223002
:1011B00042F22C0301E042F20803E3600020BDE8A4
:1011C000F08700BF455C0008C40A002000E100E091
:1011D000645E0008012838B505D80E4C14230A4473
:1011E00003FB004309E00C490320FFF7E9FC2568F5
:1011F0002D06FCD511F8015B65608A4201D01C68A0
:10120000F5E714235843034B1A5813685B06FCD5C3
:1012100038BD00BF645E0008455C00080020FFF791
:1012200051BF0120FFF74EBFF8B5104C04EB40143E
:1012300001216768384600F041F9A6680021304670
:1012400000F03CF9E5680121284600F037F9247DDB
:101250003846214600F0CEF92146304600F0CAF962
:1012600021462846BDE8F84000F0C4B9985E000861
:1012700001282DE9F041044603D910490320FFF766
:101280009FFC0F4BDFF83C80002543F820506401A1
:10129000FFF7CAFF08EB04031E7F9F6930463946FB
:1012A000FFF7C4FE58F8043039461D603046DD6152
:1012B0005D60BDE8F041FFF7DDBE00BF455C0008A2
:1012C000D40A0020985E0008012870B50C4621D889
:1012D0004A1C22D021F0FF0313F5807F11D114F0B6
:1012E000FF041AD10E4B03EB40152E69731C14D06A
:1012F0000121304600F0E2F8297D304600F07AF90D
:1013000006E00121204600F0D9F8204600F09AF9C5
:10131000002070BD4FF0FF3070BD6FF0010070BD58
:10132000985E0008042B2DE9F84304460E46154646
:10133000984603D917490320FFF742FC1648DFF807
:1013400060906701012100EB840001F0E7FC09EBEC
:1013500007031C7F99692046FFF768FE0F4B59F879
:10136000071004EB84041C4416F5807F14F8082051
:1013700045EAC20545F004050D6015BF0B684B68D2
:1013800043F4407343F0040314BF0B604B60002030
:10139000BDE8F883455C0008D40A00208C5E000894
:1013A000985E00080B4A430110B50446D018D35884
:1013B0008169007F00221A605A6822F004025A6094
:1013C000FFF758FE044800EB8400BDE8104001F030
:1013D000D5BC00BF985E0008D40A00202DE9F84370
:1013E000089E099F884691461D4623B91EB931497A
:1013F0000320FFF7E5FB304B400118F5807F1C58B8
:10140000236843F04003236005D0B8F1FF3F02D0CA
:10141000404600F020F9A6B92F44AF4206D0A36899
:101420009E07FCD515F8013B2373F6E7A3689807E0
:10143000FCD5A3681906FCD4A368DA0720D5E368B5
:10144000FAE70DB1002319E030463744B84217D00F
:10145000A3689B07FCD52573A368DE07FCD5237B17
:1014600000F8013BF2E7A2689007FCD5EA5C227322
:10147000A268D107FCD5227BF2540133BB42F2D1E2
:10148000A3689A07FCD5A3681B06FCD4B9F1000F2A
:101490000ED1B8F1FF3F0BD0236818F5807F23F001
:1014A0004003236004D04046BDE8F84300F0CAB8CA
:1014B000BDE8F883455C0008985E0008F8B50D4665
:1014C0000126C0F3832120F00F0400F00F0706FA75
:1014D00001F10220FFF7AAFD07FA06F003232168B5
:1014E00083406FEA030C01EA0C012160216805F0DA
:1014F000030E0EFA00FE4EEA01012160E2680CEADA
:101500000202E260E168C5F3810282400A43E260C0
:101510006268BE4022EA060666606268C5F300158E
:10152000BD4015436560A2681343A3600020F8BD69
:101530002DE9F04100F00F0415462B4A42F83430F3
:1015400002EBC402069B536006468846C0F383271D
:101550004FF480410120FFF769FD41463046FFF717
:10156000ADFF042C214B03DCA11D01228A4003E0C6
:10157000092C03DC4FF400021A6002E04FF4807281
:101580005A601B4B0120996800FA04F2D2431140C3
:101590009960996805EA000E0EFA04FE4EEA010110
:1015A0009960D9680A40DA60C540DA68A54004F05D
:1015B0000C0404F1804404F59C341543DD6006F00E
:1015C0000302A56892000F21914025EA0101A16064
:1015D000A1689740B0400F43A76058611A68104354
:1015E00018600020BDE8F081DC0A002000E100E086
:1015F000003C014020F00F0300F00F02F0B51E6820
:1016000057000325BD4026EA05051D601D6802241C
:10161000072A04FA07F444EA050494BF00220122D1
:101620001C6003EB820300F007001C6A80000F229D
:10163000824024EA02021A621A6A814041EA0200E8
:101640001862F0BD20F00F02012300F00F0003FA32
:1016500000F09061704720F00F0200F00F00103092
:10166000012303FA00F0906170470000104B2DE950
:10167000F0415E691A680F4F164000244FF00108D0
:101680001D4608FA04F31E4206D06B6107EBC40343
:1016900057F83420586890470134102CF1D1064B8C
:1016A0001B681BB1BDE8F041FFF7EEBABDE8F08161
:1016B000003C0140DC0A0020940200202DE9F843A0
:1016C000124ADFF8508003010746D5582E69EB68AF
:1016D00000241E4008EBC0090223A3401E4209D08B
:1016E000EA68D9F8040022EA0303EB60214658F8BF
:1016F000373098470134042CEED1054B1B681BB1E1
:10170000BDE8F843FFF7C0BABDE8F883D85E00082B
:10171000940200205C0B0020032910B516D80D4B55
:1017200000011C181B586068024001F10C0003EB1B
:10173000800042601869022202FA01F120EA0102E7
:101740001A61DA681143D960002010BD4FF0FF30F4
:1017500010BD00BFD85E00080001024B1B58586A3C
:10176000704700BFD85E0008034B00011A58136889
:1017700043F0010313607047D85E000801282DE98B
:10178000F8430546884630D81A4E1B4904013719DC
:1017900041F8302097F80C9001EBC00148464B60AF
:1017A000B968FFF743FC36597B680024346048462B
:1017B0007460F362FFF72EFC104B7A7B13F809304C
:1017C0005843B0FBF8F3013BB36251B2012302F07E
:1017D0001F02736149099340094A284642F82130A3
:1017E000FFF7C2FF2046BDE8F8834FF0FF30BDE8A9
:1017F000F88300BFD85E00085C0B0020F85E00088C
:1018000000E100E00020FFF759BF0120FFF756BFBD
:1018100070B513467BB18568C468A5420BD0846857
:101820000668651C85604568013D2C40013B345DC0
:1018300001F8014BEEE7D01A70BDC368426830B5BD
:1018400084681B1B934208D0C3680468013A5D1C7E
:101850001340C560E154002030BD4FF0FF3030BD73
:1018600013B543F25644684601F0EEFBBDF8023072
:10187000A34204D101980368DB689847F3E7024864
:1018800002F03EFEEFE700BF145F000807B571B934
:101890000C4B019043F25642B3F90010ADF8022010
:1018A000684601F0AFFB002809DC074805E0022983
:1018B00002D100F093FA02E0044802F021FE03B0E6
:1018C0005DF804FB6C0B00202C5F0008525F0008E1
:1018D00010B51A481A4CA4B002F012FEFFF778F8BF
:1018E0000121184802F082FD1749204600F076FBDE
:1018F000164B6360236820469B689847144B0293FD
:1019000000230193134B0093062208234FF4C06178
:101910001148FFF7F3F9114B0028188007DD104834
:1019200002F0EEFD802204A90E4801F0C5FE0E482B
:1019300002F0E6FD012024B010BD00BF6C5F00087E
:1019400070110020895F0008FC5E00088D180008F7
:10195000B15F0008611800086E0B00206C0B0020BE
:10196000E05F000850600008BD5F00082DE9F0410D
:101970001446274601347B78002BFAD105464FF0F8
:10198000010C974217D33C78A4F130065FFA86F831
:10199000B8F1090F07F1FF3E26D9A4F14106052E43
:1019A00002D8A4F137061FE0A4F16106052E14D871
:1019B000A4F1570618E0BCF1000F0BD1013D8542A0
:1019C00005D92A780178297000F8012BF6E7184626
:1019D000BDE8F0810020BDE8F081BCF1000FF9D135
:1019E0004FF0010C7746CCE7964518D3A7F1020ECD
:1019F00017F8017CA7F130045FFA84FCBCF1090FF1
:101A00000ED9A7F14104052C02D8A7F1370407E04D
:101A1000A7F16104052C02D8A7F1570400E00024C7
:101A200001338B42D6D846EA04142C704FF0000CD8
:101A30000135D7E77FB53823694A43439C189B5843
:101A4000014668481D6902F0D1FC022104F10E0034
:101A500000F0AEFA644802F0C9FC082104F110005D
:101A600000F0A6FAA189614802F0C0FC02230DF142
:101A7000060204212046A847002804DA5C4802F048
:101A80003FFD0120A9E0BDF806105A4802F0AEFC67
:101A900002230DF1060205212046A8470028EDDBB0
:101AA000BDF80610544802F0A1FC02230DF1060215
:101AB00011212046A8470028E0DBBDF806104F485A
:101AC00002F094FC08230DEB030219462046A847B8
:101AD000061E06DD4A4802F089FC314602A800F0E5
:101AE00067FA617E474802F081FC02230DF106028D
:101AF00026212046A8470028C0DBBDF80610424832
:101B000002F074FC02230DF1060210212046A847C2
:101B10000028B3DBBDF806103C4802F067FC022346
:101B20000DF1060224212046A8470028B4BF3848FA
:101B3000384802F0E5FC384802F058FC01230DF16A
:101B4000050212212046A847002806DD9DF8053031
:101B5000012B02D1314802F049FC01230DF10502AD
:101B600014212046A847002806DD9DF80530012BEA
:101B700002D12B4802F03AFC01230DF10502192194
:101B80002046A847002806DD9DF80530012B02D12C
:101B9000244802F02BFC01230DF105021E212046F2
:101BA000A847002806DD9DF80530012B02D11E480C
:101BB00002F01CFC01230DF105021F212046A8475D
:101BC000002806DD9DF80530012B02D1174802F0F0
:101BD0000DFC174802F094FC002004B070BD00BF5B
:101BE0007011002074600008886000089860000888
:101BF000A6600008AC600008CB600008E760000841
:101C0000F9600008106100082861000836610008CA
:101C100048610008536100085B61000865610008C5
:101C20006F610008796100087F6100088961000820
:101C3000845C000808B50020FFF7FCFE002008BD0A
:101C40002DE9F04397B006AF002304280C46BB8073
:101C500015D005281CD18A6832B1137833B102211E
:101C6000381DFFF783FE02E0104600E018460138F9
:101C700001280DD8BB885BBABB80032600E0022692
:101C8000606801F009FF54F826208046B5002AB9A3
:101C900021683E4802F0AAFB012072E01378002B75
:101CA000F6D0082107F11000FFF760FE061EEFDDF9
:101CB0002C44BB8860683B81E946B8F1000F04D032
:101CC0004146334802F092FB35E0324C3862A57E43
:101CD00002F016FE3B89786205F0280545F0010503
:101CE000A28903B93A81638BBA8103F00403002B04
:101CF000237E294903F1010E84F818E0049303952B
:101D00003B89ADF80830BB89ADF80430A1F1020081
:101D100007F12804A1F1100812BF0822014602228F
:101D2000009607F11003204601F0B6F9002804DA06
:101D30001A4802F0E5FB012022E0D8F80030F861F3
:101D4000BC611B68022207F1180140469847002831
:101D500001DA1348EDE7796A124802F047FB314691
:101D600007F1100000F024F90F4802F03FFB0221B8
:101D700007F1080000F01CF90C4802F0C1FB00203C
:101D8000CD464437BD46BDE8F08300BF90610008F2
:101D9000B96100087011002080110020D96100088D
:101DA000F9610008126200082C620008AA600008AD
:101DB0009368013B002B10B4936008DA9469A34246
:101DC00002DBCBB20A2B02D110BC02F0B3BE136807
:101DD000581C10601970C8B210BC70472DE9F04350
:101DE0005A4F5B4C0546386889B082680A21FFF774
:101DF000DFFF2B687F225E68214601AB2846B04793
:101E00008046204601F0DCF9064618B9514802F038
:101E100077FB98E003AA06A9204601F047FA02AA38
:101E2000814604A9204601F0EFF9237803F0070367
:101E30000546032B0BD8DFE803F0020406084648EA
:101E400006E0464804E0464802E0464800E04648CE
:101E500002F056FBBDF80C10444802F0C7FA4946A0
:101E600006A800F0A5F8BDF80810414802F0BEFA37
:101E7000294604A800F09CF83E4802F0B7FA2378FF
:101E800018074CBF3C483D4802F0B0FA3C4802F00D
:101E9000ADFA2378D9064CBF3748384802F0A6FA85
:101EA000384802F0A3FA23789A064CBF32483348E8
:101EB00002F09CFA344802F099FA23785B064CBF92
:101EC0003248334802F01CFB324802F08FFA617846
:101ED0003148C1F3011102F089FAA1782F4802F0CC
:101EE00085FA0022C6EB0801A01901F059FB2C4825
:101EF00002F07CFA3546C6F10109A84519D9615DA1
:101F00003868A1F120035F2B88BF3F218268FFF76B
:101F10004FFF09EB05014A23B1FBF3F203FB121358
:101F2000012B04D1AE4202D01E4802F05FFA013507
:101F3000E3E71D4802F05AFA9DF805209DF80410C9
:101F40001A4802F053FA09B0BDE8F08328020020D5
:101F5000A811002034620008576200085E62000881
:101F600075610008636200086A6200087262000816
:101F700093620008B3620008BF620008C3620008F1
:101F8000C7620008D5620008E0620008EC62000841
:101F900097630008EE620008F8620008FD6200081E
:101FA000076300080D630008835C000814630008E1
:101FB00070B5054646180446B4420AD0AC4202D079
:101FC000044802F013FA14F8011B034802F00EFA59
:101FD000F2E770BD335B00082863000810B5084BBA
:101FE0000446182240F81C3B01F0FAFF082384F84D
:101FF0003630002384F8343084F8373010BD00BF09
:102000006463000837B5044600F02AFB94F83430C6
:102010001BB90321204600F04EFA0025082168462E
:102020002576658301F09AF99DF80030019A23F036
:10203000010343F002038DF80030009B12BA1BBA73
:10204000204600F0F2F8BDF8001049BA204689B2E7
:1020500000F0DCF82046232100F018F920461A2170
:1020600000F007F92946204600F02CF9204601220D
:10207000202100F0A7F9204601224FF4807100F0E2
:10208000A1F92A4620464FF4005100F09BF9204662
:1020900001224FF4804100F095F9802220460C2166
:1020A00000F04FFA0421204600F05DFA042100F010
:1020B000FD02204600F045FA0321204600F053FAC5
:1020C000032100F0F002204600F03BFA08222046EF
:1020D0000E2100F036FA0F21204600F044FA1621B6
:1020E000204600F0E8F903B030BD10B590F8373065
:1020F0000133044680F83730204600F08CFAA0F116
:102100001103DBB2012BF7D9192818BF84F8360068
:102110001921204600F0CFF9022384F8353010BD94
:1021200070B51D4690F835306E1C1344144680F887
:10213000353013460A46F1B200F027FA601970BD37
:1021400010B5012300F135020021044600F01DFA0C
:1021500002221146204600F0F4F963683BB1628B1D
:10216000120504D520460321BDE81040184710BDD4
:10217000F8B50821044600F09EF9152107462046CF
:1021800000F0F1F960F07F02D2B215210646204638
:1021900000F0D7F90621204600F08DF908212046ED
:1021A00000F0E1F960F07F02D2B20821204600F091
:1021B000C8F90121204600F0D6F903060546F8D5F6
:1021C00032462046152100F0BCF90821204600F0D7
:1021D00072F93946204600F06EF9C5F38010F8BD5B
:1021E00038B50D460221044600F0ABF9162D07D094
:1021F000204600F010FA8542FAD184F8345038BDF8
:10220000204600F008FA1F28FAD0F6E710B50A0AAF
:1022100004468173C273202100F093F9A27B20460B
:102220002121BDE8104000F08CB92DE9F8430546A6
:1022300016461F4600F10F0800246FF00709E20060
:102240003046394601F01CFC09FB04F208F8010F86
:1022500038323046394601F013FC04F12401C2B291
:10226000C9B22846013400F06CF9082CE7D1BDE86A
:10227000F883A1F10B020F2A05D8427E8A4202D0D0
:10228000417600F009BA70470020704737B50D0A53
:102290008181CAB22221044600F053F92A46232143
:1022A000204603B0BDE8304000F04BB908B5052129
:1022B00000F059F9024B00F00F0033F9100008BD8F
:1022C00042630008113109B21429A8BF142121EA80
:1022D000E171024B5A5C052100F033B92D6300080F
:1022E00008B52C2100F03FF9C0F3071008BD38B540
:1022F0000C462C21054600F036F9072C28BF072490
:1023000000F00F0040EA0412D2B228462C21BDE8AA
:10231000384000F016B908B52C2100F024F9C0F3BC
:10232000420008BD0529A8BF0521002938B50C4683
:10233000A8BF0C464FF02C010546B8BF072400F09B
:1023400012F920F00E0040EA4402D2B228462C21B5
:10235000BDE8384000F0F5B838B505460C4699B1EF
:102360000A782D2100F0EDF82E21284600F0FBF828
:10237000637800F0F80203F007031A4328462E2181
:10238000BDE8384000F0DDB838BD08B5092100F0DF
:10239000EAF800F00F0040005B3840B208BD0029A9
:1023A000C4BF494249B25B31C1F3430242F0C002AB
:1023B000092100F0C6B808B5072100F0D4F85B3851
:1023C00040B208BD10B5438B0446B2B30B43B1F520
:1023D000807F43830AD002D8202925D010BDB1F5D3
:1023E000007F0ED0B1F5005F20D010BD00F11001CC
:1023F000FFF7B2FF04212046FFF794FF53222F215D
:1024000053E02E2100F0AFF840F01002D2B22E219E
:10241000204600F096F81721204600F0A4F840F07E
:102420000202D2B2172140E02E212BE00E2100F053
:102430009AF840F00402D2B236E023EA0103B1F583
:10244000807F43830AD002D8202921D010BDB1F566
:10245000007F09D0B1F5005F21D010BD4FF0FF31F2
:10246000BDE81040FFF75EBF172100F07CF8172190
:1024700000F0FD02204600F064F8638B9B0619D53E
:102480002E21204600F06FF800F0EF022E210CE024
:102490002E2100F068F840F01002D2B2F6E70E21CB
:1024A00000F061F800F0FB020E212046BDE810406C
:1024B00000F047B810BD70B504460D46204600F048
:1024C000AAF8A0F11103DBB2012B0646F6D91F28AA
:1024D000F4D0032D02D12A46082126E0A84227D0B5
:1024E000162801D1192D02E0192807D1162D0AD17D
:1024F000092211462046FFF773FE04E00F2802D19F
:10250000204600F094F80F2D0DD103212046FFF74F
:10251000D2FF2946204600F026F8E06AFFF792F83D
:1025200084F8345004E02A4629462046FFF758FE36
:10253000304670BD90F82030416AC0690022FEF735
:10254000F1BE70B504460D461646FFF7F3FF33465D
:1025500045F0C002616AE06901F06BF8E069BDE82E
:102560007040FEF71FBF38B504460D46FFF7E2FF87
:1025700045F080020023616AE06901F05AF80546DF
:10258000E069FEF70FFF284638BDF7B504460F4651
:1025900015461E46FFF7CEFF616AE069402301221F
:1025A00001F036F83B46616AE069012201F030F83B
:1025B0000022E069019600922B46616AFEF70EFF49
:1025C000E06903B0BDE8F040FEF7ECBE10B504468C
:1025D000FFF7B0FF616AE06920230122BDE81040E7
:1025E00001F016B807B58DE806000023416AC069FE
:1025F0000122FEF7F3FE03B05DF804FB10B50446BC
:10260000416AC0690123002201F002F8E069BDE8D7
:102610001040FEF7C7BE08B590F834300F2B04D039
:102620000121FFF7A0FF00F01F03184608BD10B5F9
:102630000446FFF7F0FF0F2811D1E06AFFF70BF80F
:1026400000214FF4997001F07DF901212046FFF738
:102650008AFF00F01F00082884F83400F5D110BD6F
:1026600010B50446006BFEF7F6FF00213E2001F096
:1026700069F9206BFEF7E6FF00213E2001F062F9C8
:1026800001212046FFF76FFF00F01F0310F0170F26
:1026900084F83430F4D110BD38B508210446FFF772
:1026A0000AFF082105462046FFF75DFF637E00F024
:1026B000E00203F01F0320461A430821FFF741FF01
:1026C00029462046BDE83840FFF7F5BE43680BB108
:1026D00000211847704700002DE9F047044688465E
:1026E00016461F46FFF797FF8146002C00F0D38067
:1026F0000F2840F0DF80B8F1180F66D02046FFF7B2
:1027000096FFB8F1270F00F22B81DFE818F04200A6
:10271000290128003300290129013B002901290151
:10272000290129012901290129012901290155002E
:1027300029018B008F007E002901840029012901D5
:102740002901930097009B009F002901A300AA0084
:10275000290129012901290129014E00BA00022F6E
:1027600003D98B490320FEF72BFA31882046FFF767
:102770004DFD94E0082FF4D8D6E900232046FFF75A
:1027800054FD8CE0022FECD831882046FFF77EFD07
:1027900085E0012FE5D03178A1F10B030F2B00F27A
:1027A000EC802046FFF765FD79E0012FD9D0337822
:1027B000002B40F0E2806CE0022FD2D8B6F9001076
:1027C0002046FFF77FFD0225D9E0012FC9D83378D5
:1027D000013B052B63D8DFE803F00507620C140307
:1027E000082102E00F2100E016212046FFF763FEDA
:1027F000CBE0638B5A0540F1C8802046FFF7A0FC70
:10280000C3E02046FFF7FEFBBFE0327820212046E0
:10281000FFF7D8FD43E0012FA3D831782046FFF71A
:1028200066FD36E032784FF4806116E032784FF47E
:10283000007112E032784FF400510EE032784FF41C
:1028400080410AE032784FF4006106E032784FF4BC
:10285000805102E032784FF480712046FFF7B2FDDC
:1028600017E0012F3FF67DAF638BDB0503D4337890
:10287000052B40F2828096F900102046FFF752FDAA
:1028800007E0012F3FF66DAF96F900102046FFF7E5
:1028900086FD012573E06FF01200BDE8F087B9F105
:1028A0000F0F5DD03B46324641462046BDE8F0471B
:1028B00000F002BEB8F1270FF4D801A353F828F0B6
:1028C00093270008A52800085F270008752700083F
:1028D000A5280008A528000885270008A5280008C5
:1028E000A5280008A5280008A5280008A528000894
:1028F000A5280008A5280008A5280008A528000884
:10290000B9270008A5280008252800082D28000858
:102910000B280008A528000817280008A52800088B
:10292000CB270008A5280008352800083D28000806
:10293000452800084D280008A5280008552800084B
:1029400063280008A5280008A5280008A528000875
:10295000A5280008A5280008AB2700088328000840
:10296000B8F1180F9ED06FF085050F212046FFF7B4
:10297000A2FD15F1860F05D194E76FF01505B9F1A9
:102980000F0FF2D02846BDE8F0870120BDE8F087A0
:10299000455C00082DE9F0410446FFF73CFE0F2896
:1029A00006464CD00F212046FFF7DDFD02210746E9
:1029B0002046FFF7D8FD7B07054603D56368012154
:1029C0002046984738073AD5162E01D0112E05D14A
:1029D000638B590433D5636802212CE0192E01D092
:1029E000122E2CD194F837301BB916490320FEF76C
:1029F000E7F8013BDBB284F8373023B994F836109E
:102A00002046FFF758FD6368CBB1628BD20416D520
:102A100005F0E000202809D002D838B1BDE8F081E7
:102A2000602807D0A02803D0BDE8F081042102E08F
:102A3000062100E007212046BDE8F0411847BDE827
:102A4000F08100BF455C000813B50446416AC069C7
:102A5000FEF73AFC0121E06AFEF730FDE06AFEF77E
:102A6000FAFD0121206BFEF729FD206BFEF7EAFD40
:102A7000094B009401220021A06AFEF759FD20466F
:102A8000FFF7C0FA1C212046FFF76DFD033818BF81
:102A90004FF0FF3002B010BDCD2600082DE9F34104
:102AA00004460F4690461E46FFF790FD01220DF1A9
:102AB00003012046FFF796FD9DF8035005F07F05C2
:102AC000023D07B3454505D92046FFF797FD6FF056
:102AD00068051BE02A4639462046FFF783FD02229F
:102AE00001A92046FFF77EFD6EB10122B1182046F4
:102AF000FFF778FD2046FFF781FD07212046FFF70D
:102B000032FD307002E02046FFF778FD284602B023
:102B1000BDE8F0812DE9F04107460D469046FFF7EC
:102B2000E4FA0026344646450FD06A68A31C1344D5
:102B30007F2B05F1080511D8234655F8081C3846A7
:102B4000FFF7EEFA01360446EDE77B8B5B0502D416
:102B50003846FFF7F5FA2046BDE8F0816FF08A00AD
:102B6000BDE8F08108B5FFF756FD0838C0B211285E
:102B70009ABF024B185C022008BD00BF7C630008AE
:102B80002DE9F8430F46164698460546002800F002
:102B9000B780A1F11103152B4DD8DFE803F01827FA
:102BA000344C4C4C4C204C383C40444C484C4C4CE5
:102BB0004C4C4C0BB8F1010F03D857490320FDF7DB
:102BC000FFFF00237370FFF75FFB307004E0B8F184
:102BD000010FF2D9662333800220BDE8F883B8F1F3
:102BE000000FEAD0FFF7BEFF307009E0438B13F40B
:102BF000806F03D001203070BDE8F883002333706C
:102C00000120BDE8F883438B13F4007FF1E7438B89
:102C1000C3F34033F3E7438BC3F38033EFE7438BD6
:102C2000C3F3C023EBE7438BC3F30033E7E7438BE6
:102C3000C3F30023E3E74346324600F09DFB10F167
:102C4000860F044660D12846FFF7E5FC0F28814631
:102C500011D12846FFF7EBFC162F1CD004D8012F0A
:102C600035D0102F0ED046E0272F28D02F2F36D06A
:102C7000202F1DD03FE0162F0DD013D8012F26D0C6
:102C8000102F44D1B8F1010F97D92846FFF70EFB5A
:102C9000022430802CE0B8F1000F8ED02846FFF7D8
:102CA0001FFB23E0272F0AD02F2F18D0202F2ED143
:102CB000B8F1000F81D02846FFF72DFB16E0B8F1E0
:102CC000000F3FF47AAF2846FFF75FFB0EE0B8F144
:102CD000000F3FF472AF2846FFF74AFA06E0B8F15A
:102CE000000F3FF46AAF2846FFF765FB3070012400
:102CF000B9F10F0F08D10F212846FFF7DCFB03E0E5
:102D00006FF01200BDE8F8832046BDE8F8836FF04D
:102D10008500BDE8F88300BF455C000870B5054636
:102D20000C46FDF79DFB2B6806462BB94FF0FF3391
:102D30002B60FDF79DFB18E0CCB10F4B1C68022106
:102D40002046FDF793FA2B68013305D104F10803FF
:102D50002B600023A36003E021462846FDF7AEFF69
:102D60003046FDF785FBFDF757FB012070BDFDF7F1
:102D70007FFB204670BD00BF9C02002070B504465A
:102D8000FDF76EFB256806461DB16B1C05D10023BF
:102D90002360BDE87040FDF76BBB28460A2150F860
:102DA00008392360FDF762FA236813B94FF0FF3347
:102DB000236015F8034C3046FDF75AFB2046BDE86A
:102DC0007040FDF793BA0000F8B505460E46FDF7D2
:102DD00047FB364B364A1B881BB2074652F8232066
:102DE000D2F820E0BEF1000F1AD054699369A342D3
:102DF00016D9631C5361D3691C4046B9136933B9B2
:102E0000631C04D13846FDF733FB2046F8BD002C87
:102E10000ADB0EEBC40393E8030085E8030004E03B
:102E20004FF0FF34002EE9D0D560166976B33368D1
:102E30001361002C0CDB95695169D369691A8B42C7
:102E4000A9BF691C4FF0FF351D4091610EEBC50510
:102E5000736893E8030085E8030016F8043C052B2B
:102E600009D0002373600A21A6F10800FDF7FEF9DE
:102E700016F8034C00E00F243846FDF7F9FA0E2C43
:102E800002D82046FDF732FA0120F8BD002C09DAFD
:102E900010460321FDF7EAF93846FDF7E9FAFDF798
:102EA000BBFAF1E73846FDF7E3FAEDE798020020B8
:102EB000E402002010B583694469C2691C1BA24268
:102EC00001DA002010BD5C1C13408461F9D4026A51
:102ED00003C902EBC30383E80300012010BD000017
:102EE0002DE9F8431E46264B53F82150254B1B88ED
:102EF0000380074691462DB93046FDF7B9FA4FF0E9
:102F0000FF3439E02B79032B28D01F4B014628468C
:102F1000D3F80080FFF7CEFF044638B13046FDF706
:102F2000A7FA98F80430052B25D122E0B9F1000F5B
:102F300003D13046FDF79CFA1EE098F80430C8F83B
:102F40000C70052B0CBF052104214046FDF78EF9BE
:102F5000414605F11000FDF7B1FE07E003C8EB683C
:102F600083E803000A212846FDF780F93046FDF783
:102F70007FFAFDF751FA01242046BDE8F88300BF2F
:102F8000E4020020980200209C02002038B504468C
:102F9000FDF766FA074B1B882380074B2146054641
:102FA0001868FFF787FF04462846FDF761FA2046B8
:102FB00038BD00BF980200209C02002008B50F4BCE
:102FC00053F82130B3B1212202801A79032A0BD1A0
:102FD00003C8DA6882E8030018460A21FDF746F9BB
:102FE000074B0120186008BD01461846BDE808409F
:102FF000FFF760BF4FF0FF3008BD00BFE4020020C4
:103000009402002070B504460D46FDF734FA28B14D
:1030100029462046BDE87040FFF7D0BF094B1B880A
:103020001BB29D4204D12046BDE87040FFF7AEBF01
:10303000FDF716FA2946034601222046BDE87040F6
:10304000FFF74EBF980200200121FFF7BDBE000030
:103050000F4BD3F8882042F47002C3F888200D4A41
:103060009A60102283F822200021DA7701F1604073
:1030700000F561400131522980F80023F6D11A6928
:1030800042F010021A615A6942F400725A617047A4
:1030900000ED00E000000008F8B504469DF824505B
:1030A00025701E4605F0070310250F46657006982B
:1030B0009DF8281015460AB1002F68D018B1002ECF
:1030C00069D13046F8BD23B1022B02D00DB90028DA
:1030D00073D0A17080B39DF82030E37002289DF872
:1030E0002130237104D0082816D0002851D120E0C7
:1030F00002463249304600F041FF18B9237823F0E8
:1031000020032370637843F008036370737863715E
:103110003378A371072040E01C236370221D06F161
:10312000080313F8011D02F8011F9E42F9D10D207A
:1031300033E005201DB9F8BD0320002D3DD0431C10
:103140009DF81C2022549DF81D20E2540230022DCF
:1031500003D0082D0CD0E5B9F8BD637863F07F0388
:1031600063707A782254431C3A78E2540230F8BDF6
:10317000637863F03F03637007F10803044413F8B6
:10318000012D04F8012BBB42F9D10830F8BD3846B7
:10319000F8BD0020F8BD63B90DE075B1BDF81C2085
:1031A000BDF820309A42CAD1237843F040032370FF
:1031B000CDE7022B8AD1A1708DE7F8BD8E630008A0
:1031C000427802F00C03082B07D00C2B07D0CBB9A8
:1031D0000178490614D4032302E0072300E00D23FD
:1031E00012F0C0020CD00178490658BF0233802A81
:1031F00001D1981C7047C02A04D103F10800704720
:10320000184670470020704770B501B11AB92649B9
:103210000320FDF7D5FC437803F00C03082B07D1FE
:1032200003785C0617D5C37813700379537012E0E6
:103230000C2B07D103785B060FD5C3781370037985
:1032400053700AE013B16FF0150070BD03785E068D
:10325000F9D4032302E0072300E00D23447814F09F
:10326000C00411D005786D0605D4C65C16705D1CCF
:103270000233455D5570802C08D1C25C4A7003440E
:1032800002205B780B7070BD204670BDC02CDAD177
:10329000034401F1080213F8010B02F8010D8A4200
:1032A000F9D1082070BD00BF455C000808B501B128
:1032B0001AB918490320FDF783FC437803F00C0387
:1032C000082B09D1C37813700379537043794B707D
:1032D00083790B70022008BD0C2B0ED1C3781370BC
:1032E00010F8043F537001F1080310F8012F03F8A0
:1032F000012D8B42F9D1082008BD3BB9037813F0AA
:10330000400F14BF6FF01500002008BD6FF01500CE
:1033100008BD00BF455C00087FB50C46054600B1FE
:1033200019B90D490320FDF74BFC0A4601AE2321D4
:1033300000F054FF304600F065F90023B3FBF4F2CF
:1033400004FB1232F15CA85C013341400C2BA95400
:10335000F4D104B070BD00BF455C000810B5044650
:10336000FFF7DAFF034B1A78511C1970237853408A
:10337000237010BD24020020052938B50C461546DF
:1033800006D8042928D202290FD01CD899B38BE083
:10339000152935D004D8062928D0082947D083E03C
:1033A00019293AD025293ED07EE0012B03D8414986
:1033B0000320FDF705FC0A4600F10E01284600F047
:1033C0000FFE204638BD072BF1D900F1100108226D
:1033D000284600F005FE6AE0022BE8D1428B520736
:1033E00001D5082205E02B80184638BD022BDED11E
:1033F00082892A80F8E7022BD9D1437E13800AE024
:10340000012BD4D1438B13F0200F02D001232B705A
:10341000EAE700232B70012038BD012BC7D1438B75
:1034200013F0020FF1E7022BC1D10322E1E7072BD2
:10343000BDD9438B5B074CBF0B4602234FF0000204
:103440004CBF10300E30042B6A702A7018D0082B35
:1034500003D0022B2BD1134619E0027882F002022E
:103460002A7042786A708278AA70C278EA7002790B
:103470002A7142796A718279AA71C279EA71B3E7D5
:10348000037883F002032B7043786B700223FF21D3
:103490000022E970FE21AA7029716A71C25CAA71CA
:1034A00018444378EB7102E06FF0850038BD0820C6
:1034B00038BD00BF455C00080529F8B50D46164625
:1034C0001C4606D8042936D2022914D023D839B193
:1034D0005DE0152947D019294ED0062957D13CE087
:1034E000022B03D02D490320FDF76AFB1388FF2B25
:1034F000F8D8437635E0022BF4D800F10E070A46DF
:103500003846002100F06AFE22463146384600F077
:1035100067FD2846F8BD082BE4D800F11005082205
:103520000021284600F05AFE22463146284600F087
:1035300057FD0820F8BD022BD4D11388022B06D0EA
:10354000082B27D1438B43F00403438309E0428BCC
:1035500022F0040242831846F8BD022BC2D1138820
:1035600083812046F8BD1278438B12B143F02003CB
:103570000AE023F0200307E01278438B12B143F0F6
:10358000020301E023F0020343830220F8BD6FF041
:103590008500F8BD6FF06900F8BD00BF455C00080C
:1035A0002DE9F8431546814613480F4600F05EFAB0
:1035B000002D08BF1025002407F1FF38A74218D0BE
:1035C0000E4800F053FA661C19F8040000F036FAB1
:1035D000B6FBF5F305FB13630BB1A04507D1084813
:1035E00000F08EFFA04502D0304600F033FA34469A
:1035F000E4E7BDE8F88300BF9063000811630008AA
:10360000845C00080C22014900F0EABC107AFF1F1C
:1036100010B586B006AC04F8093D012301930DF105
:10362000170300932346FDF7D9FE9DF8170006B057
:1036300010BDF0B585B01F4604AB002403F8012D82
:10364000012205460E4601920094FDF7C7FE3B4657
:10365000224631462846FFF7DBFF05B0F0BD0000EB
:103660000C4B0146186882689368013B002B10B42C
:10367000936005DA9469A34208DBCBB20A2B05D02C
:103680001368581C1060197010BC704710BC01F012
:1036900051BA00BF2802002008B53E20FFF7E0FF26
:1036A0002020FFF7DDFF034B1B689868BDE808404A
:1036B00000F0C4BA280200202DE9804885B0814678
:1036C00000AF0E469246FFF7E7FFB0460AF1FF341F
:1036D0000025C6EB0803A342F5DA844B186841685D
:1036E0004B68013B002B4B6004DA00F011FF00280F
:1036F00004DAE8E70B685A1C0A6018780D2801D034
:103700000A280FD100240D2088F80040FFF7A8FFF9
:103710000A20FFF7A5FF4645D5D033462246254669
:1037200020462BE0082801D07F280DD14645D0D077
:10373000082008F8015CFFF793FF2020FFF790FFB7
:1037400008F1FF3B082003E008F1010B88F80000B6
:10375000FFF786FFD846BCE7222913D15C781CB35B
:103760005C2C25D001331C788C42F7D15978202964
:103770001AD80135197811B303F8010B19782029EB
:10378000F8D9E9E7272906D1E8E74B1C497822292F
:103790000AD02029EDD91C785C2C1946F5D1591C8A
:1037A0005B780132002BF0D1514800F0A9FE8AE786
:1037B0009C1C9B780132002BF6D02346D3E7002DCA
:1037C00081D0AB000E3323F00703EB46ADEB030DC6
:1037D0006C464DF82510304690F800E00346013065
:1037E000BEF1000FF8D0BEF1220F02D0BEF1270FBC
:1037F00000D1013344F821301846013390F800E03D
:10380000BEF1000FF8D101318D42E5D1201FBAB1D0
:1038100050F8043FA3B1194613F801EBBEF1000FB5
:10382000F5D0BEF15C0FF6D191F800E0BEF1000FCB
:1038300004D091F801E001F801EBF5E7013AEAD193
:103840002C4B2268FB60C7F80890002307F10801A1
:1038500051F82380B8F1000F0DD10133022B16D09F
:10386000F4E711463B607A6000F0DEFE7A683B6860
:1038700030B108F10C08D8F800000028F1D1ECE7CD
:10388000D8F808301BB12146284698472CE021681B
:10389000194800F0C9FE054610BB184A18491948D6
:1038A00000F0A4FD184800F02BFE124BC7F808905A
:1038B000FB602C4607F1080353F824500DB10C357A
:1038C00003E00134022CF5D10EE00C3555F8181C3C
:1038D0000029F6D055F8142C0A4800F087FDF4E7CB
:1038E00021680A4800F082FDDD46ECE6280200204F
:1038F0009963000860640008B2630008B7630008B9
:10390000C3630008CB630008D5630008FD630008AB
:1039100008B500F041F8002008BD08B5FDF7B0FA81
:10392000002008BDFFF72ABA38B504460020FDF78D
:1039300013FF05460020FDF70FFF401BA042F9D3FF
:1039400038BD000030B587B004460D46FCF793FD46
:1039500040B11DB10E490320FDF732F92046FFF7B3
:10396000E3FF13E00B4B00900390029001216846A7
:103970000493CDF814D0FFF7D1F9214601A82A46C7
:10398000FDF7CCF801216846FFF7C8F907B030BD54
:10399000455C000825390008BFF34F8F0549064BE9
:1039A000CA6802F4E0621343CB60BFF34F8F00BFDD
:1039B000FDE700BF00ED00E00400FA0538B1054B5B
:1039C0000A0901F00F019A5C5B5C027043700220EF
:1039D000704700BF8464000803461A78591C0AB176
:1039E0000B46FAE7181A7047F8B505460F46164613
:1039F0008C18BC4206D0284614F8011DFFF7DEFFE4
:103A00000544F6E77000F8BD07B502AB042243F8A1
:103A1000041D1946FFF7E8FF03B05DF804FB38B555
:103A200005460C464CB122462946012001F076F8A5
:103A3000002802DB241A0544F4E738BD07B5014627
:103A400001A8FFF7BBFF022101A8FFF7E8FF03B0C1
:103A50005DF804FB07B501466846FFF7D5FF08216E
:103A60006846FFF7DCFF03B05DF804FB10B50446C1
:103A7000FFF7B2FF01462046BDE81040FFF7CFBF79
:103A8000D0400B1CD1409C46203AD34018435242B0
:103A900063469340184370470A22002101F032B870
:103AA0000A23002200F09ABF8B891A072DE9F04102
:103AB0000D46804635D44A68002A6BDDEC6A002C3E
:103AC00047D003F48052002192B2D8F80060C8F8C1
:103AD0000010002A62D06A6D5F0705D569686B6BBC
:103AE000521A0BB12B6CD21A0023296A4046A04708
:103AF000441C39D0AB892A692A60DB044FF00002EC
:103B00006A6045D4696BC8F8006011B305F14403DD
:103B1000994202D0404600F0AFFB00206863BDE848
:103B2000F0810E69AEB10C680E6098070CBF4B694E
:103B30000023A41B8B600AE023463246AF6A296A41
:103B40004046B8470028A4EB0004064404DD002CDE
:103B5000F2DC0020BDE8F081AB8943F04003AB818B
:103B60004FF0FF30BDE8F081D8F800201D2AF3D8CF
:103B7000184BD34003F0010383F00101002BEBD07D
:103B8000AB892C696960D9042C60BBD5002AB9D1F6
:103B90006865B7E70A6C002A90DCDAE70123296A36
:103BA0004046A047431C024602D0AB89EC6A93E72B
:103BB000D8F80030002BF8D01D2B01D0162B02D1E5
:103BC000C8F80060C5E7AB8943F04003AB81BDE8AE
:103BD000F08100BF010040200B6933B310B50446EB
:103BE00082B008B18369ABB1114B994219D0114B26
:103BF000994218D0104B994208BFE168B1F90C30D6
:103C000013B9002002B010BD204602B0BDE810403C
:103C1000FFF74ABF019100F019F90199044B99424D
:103C2000E5D16168EAE7A168E8E70020704700BFD6
:103C3000D4640008B46400089464000820B1054B03
:103C400001461868FFF7C8BF034B0449186800F025
:103C500043B900BF28020020F4640008D93B0008E3
:103C600000207047014900F037B900BFD93B000878
:103C70000020704770B568234D1E03FB05F50E4606
:103C800005F1740100F03EFB044640B100210C3008
:103C9000666005F168022160A06000F09FFA20468E
:103CA00070BD00BF1F4B70B51D68AB69064613B9E8
:103CB000284600F039F848356B68AC68013B05D5FB
:103CC00021E0013B5A1C04F168041CD0B4F90C201B
:103CD000002AF6D1002501234FF6FF72E281A3816D
:103CE00065662560A560656025616561A5612946F9
:103CF000082204F15C0000F071FA6563A563A56415
:103D0000E564204670BD2B680BB11D46D4E7042145
:103D10003046FFF7AFFF286008B10546CCE70C231B
:103D2000336070BDF46400083D4B3E491A682DE9CC
:103D3000F04F90424FF000038364C364036508BFF3
:103D4000012383B008BF836181620746FFF7AAFFA2
:103D500078603846FFF7A6FFB8603846FFF7A2FF45
:103D60007D68F86000240423AB812C606C60AC603B
:103D70006C66EC812C616C61AC61214605F15C00E4
:103D8000082200F02BFABE68DFF89CB0DFF89CA098
:103D9000DFF89C90DFF89C80C5F824B0012309224D
:103DA000C5F828A0C5F82C90C5F830802D622146B2
:103DB000F381B28134607460B4607466346174619C
:103DC000B46106F15C000822019300F007FAFD6877
:103DD000366212200222C6F824B0C6F828A0C6F81F
:103DE0002C90C6F830802146A881EA812C606C6056
:103DF000AC606C662C616C61AC6105F15C00082202
:103E000000F0ECF9019B2D62C5F824B0C5F828A09C
:103E1000C5F82C90C5F83080BB6103B0BDE8F08FC9
:103E2000F4640008653C000881450008A9450008C5
:103E3000E545000805460008024B0349186800F0F4
:103E40004BB800BFF4640008D93B0008836903B98C
:103E50006AE77047704700BF704700BF704700BFF8
:103E6000704700BF024B0349186800F00FB800BF4D
:103E700028020020713C0008024B0349186800F03A
:103E800005B800BF28020020613C00082DE9F04180
:103E900010F148071BD0884600267D68BC68013DAC
:103EA0000FD4A389012B05F1FF3506D9B4F90E30E3
:103EB0000133204601D0C04706436B1C04F168045F
:103EC000EFD13F68002FE8D13046BDE8F0813E4693
:103ED0003046BDE8F08100BF2DE9F84310F14807F6
:103EE0001FD0884606464FF000097D68BC68013D3A
:103EF00011D4A389012B05F1FF3508D9B4F90E308F
:103F000001332146304602D0C04749EA00096B1C04
:103F100004F16804EDD13F68002FE6D14846BDE8C2
:103F2000F883B9464846BDE8F88300BF70B50F4E28
:103F30000F4D761BB61018BF002405D0013455F87C
:103F4000043B9847A642F9D10A4E0B4D761BFCF76D
:103F50001DF9B61018BF002406D0013455F8043BF3
:103F60009847A642F9D170BD70BD00BF3C660008FD
:103F70003C6600083C6600083C660008032A70B4F2
:103F800026D940EA01039B0711D004780D78AC4292
:103F900022D10244431C05E013F8014B11F8015FE4
:103FA000AC4219D19342F7D1002070BC70470C4647
:103FB00003461E682568AE421846214603F10403F5
:103FC00004F10404E1D1043A032A18462146F0D84A
:103FD000002ADAD11046E8E7601B70BC704700BFCA
:103FE000844641EA000313F003036DD1403A41D304
:103FF00051F8043B40F8043B51F8043B40F8043BC3
:1040000051F8043B40F8043B51F8043B40F8043BB2
:1040100051F8043B40F8043B51F8043B40F8043BA2
:1040200051F8043B40F8043B51F8043B40F8043B92
:1040300051F8043B40F8043B51F8043B40F8043B82
:1040400051F8043B40F8043B51F8043B40F8043B72
:1040500051F8043B40F8043B51F8043B40F8043B62
:1040600051F8043B40F8043B51F8043B40F8043B52
:10407000403ABDD2303211D351F8043B40F8043BF2
:1040800051F8043B40F8043B51F8043B40F8043B32
:1040900051F8043B40F8043B103AEDD20C3205D302
:1040A00051F8043B40F8043B043AF9D2043208D0FA
:1040B000D2071CBF11F8013B00F8013B01D30B886C
:1040C00003806046704700BF082A13D38B078DD04A
:1040D00010F003038AD0C3F10403D21ADB071CBF1C
:1040E00011F8013B00F8013B80D331F8023B20F886
:1040F000023B7BE7043AD9D3013A11F8013B00F8BF
:10410000013BF9D20B7803704B7843708B78837046
:10411000604670478842F0B50DD98B1898420AD294
:104120008118002A51D09A1A13F8014D01F8014D57
:104130009342F9D1F0BD0F2A48D941EA00039B0709
:1041400046D100F1100401F11003154653F8106C2C
:1041500044F8106C53F80C6C44F80C6C53F8086C71
:1041600044F8086C103D53F8046C44F8046C0F2DAF
:1041700003F1100304F11004E8D8A2F1100323F0B6
:104180000F0302F00F0E1033BEF1030F1944034466
:1041900021D91E1F0D467446043C55F8047B46F891
:1041A000047F032CF8D8AEF1040424F00304043493
:1041B0002344214402F0030262B1013B0A4411F896
:1041C000014B03F8014F8A42F9D1F0BD0346F3E7F2
:1041D0000346F2E7F0BD7246EEE700BF70B4840715
:1041E00046D0541E002A41D0CDB2034602E0621EE2
:1041F000E4B3144603F8015B9A07F8D1032C2ED9D7
:10420000CDB245EA05250F2C45EA054519D903F13C
:1042100010022646103E0F2E42F8105C42F80C5C4D
:1042200042F8085C42F8045C02F11002F2D8A4F1F2
:10423000100222F00F0204F00F041032032C13447A
:104240000DD91E462246043A032A46F8045BFAD8E2
:10425000221F22F003020432134404F003042CB1A1
:10426000C9B21C4403F8011BA342FBD170BC7047C8
:1042700014460346C2E700BF30B481B151F8043C94
:104280000439002BB8BFC9181D4B1A682AB18A42DD
:104290000AD908680C18A24225D04A60196030BCBF
:1042A00070478B4203D81A465368002BF9D1146823
:1042B00015198D420CD007D808680C189C4218D0EC
:1042C0004B6030BC516070470C23036030BC7047BA
:1042D00009680C44111999421460E0D10ACB0C44CE
:1042E00053601460DBE7146852684A602044086039
:1042F000D4E71C685B684B60204408605160CEE7DF
:104300002812002070B5CD1C25F0030508350C2DB2
:1043100038BF0C25002D06463BDBA94239D827497A
:104320000A6852B113685B1B04D436E023685B1B38
:104330001AD522465468002CF8D149681F4C002930
:1043400036D029463046FBF725FF431C21D0C41C3C
:1043500024F00304A04205D0211A3046FBF71AFFCF
:10436000013016D0256004E00B2B0DD923601C44CE
:10437000256004F10B0020F00700231DC31A02D0B2
:104380005A42E25070BD70BD94420ED063685360D3
:10439000EFE70C233360002070BD0B2B03D853686C
:1043A00014460B60E5E71446E0E713461446F8E7C9
:1043B0003046FBF7EFFE6060C3E700BF2812002025
:1043C0000EB410B5044683B018B183690BB9FFF77A
:1043D0003DFD06A803460190059AA168204600F01D
:1043E00033FD03B0BDE8104003B070470FB410B503
:1043F0000A4B1C6882B024B1A36913B92046FFF7A9
:1044000025FD05A803460190049AA168204600F006
:104410001BFD02B0BDE8104004B070472802002028
:104420002DE9F0410E46804600283ED08369002BDE
:1044300039D084682F4B9C4243D02F4B9C4256D09E
:104440002E4B9C4208BFD8F80C40A3891B073DD5D2
:104450002369002B3AD0013EA36816F8015F013BA7
:10446000A360B5B1002B04DB23685A1C22601D70C9
:10447000F2E7A769BB4222462946404601DB0A2DE6
:10448000F2D100F057FB0130E6D14FF0FF30BDE82C
:10449000F081002B21DB23680A22591C21601A704D
:1044A0001046BDE8F081FFF7D1FCD8F81830D8F8F5
:1044B0000840002BBED14046FFF7C8FC0D4B9C4284
:1044C000BBD1D8F80440A3891B07C1D4214640467C
:1044D00000F092FB0028BED0D7E7224640460A21D2
:1044E00000F028FB0130D0D00A20BDE8F081D8F8D8
:1044F0000840AAE7D4640008B46400089464000883
:10450000024B01461868FFF78BBF00BF280200204E
:1045100038B50C46054608B18369B3B1114B9C42CE
:1045200018D0114B9C4217D0104B9C4208BFEC682E
:104530002846214600F0BEFF80B994E80C00013BFC
:10454000511C84E80A00107838BDFFF77FFC054B4A
:104550009C42E6D16C68EBE7AC68E9E74FF0FF30CE
:1045600038BD00BFD4640008B46400089464000837
:10457000024B01461868FFF7CBBF00BF280200209E
:1045800010B50C46B1F90E10FBF722FE002803DB34
:10459000636D0344636510BDA38923F48053A38135
:1045A00010BD00BF002070472DE9F0411646B1F95B
:1045B0000C201F46D3050C46054607D500220223D2
:1045C000B1F90E10FBF711FEB4F90C20B4F90E107E
:1045D00022F48052A2813B4632462846BDE8F04193
:1045E000FBF7FABD10B50C46B1F90E10FBF7FDFD57
:1045F000A389421C0EBF23F4805343F480536065AB
:10460000A38110BDB1F90E10FBF7EABD0000000058
:10461000000000000000000000000000000000009A
:10462000A2EB0300704700BF02780B78012A28BF75
:104630009A42F5D16DE9044540EA0104CDE90267EB
:104640006FF0000C4FEA447212B380EA010414F0D8
:10465000070F6AD100F0070420F0070004F00305FB
:1046600021F007014FEAC505F0E8042314F0040F18
:10467000F1E804670CFA05F462EA040266EA04064B
:104680000AD063EA0403624667EA0407664603E069
:10469000F0E80423F1E8046782FA4CF582EA0604A4
:1046A000A4FA8CF46CBB83FA4CF583EA0705A5FAEF
:1046B0008CF595B950E9022351E9026782FA4CF56D
:1046C00082EA0604A4FA8CF483FA4CF583EA07051F
:1046D000A5FA8CF52543DBD09CB92DBAB5FA85F443
:1046E00024F0070427FA04F1DDE9026723FA04F352
:1046F00003F0FF0001F0FF01FDE80445A0EB01001D
:10470000704724BAB4FA84F424F0070426FA04F1BA
:10471000DDE9026722FA04F202F0FF0001F0FF0176
:10472000FDE80445A0EB0100704714F0030F3CD1F5
:1047300010F0030428D150F8082B51F8083B82FAF6
:104740004CF582EA0305A5FA8CF55DB950F8042C06
:1047500051F8043C82FA4CF582EA0305A5FA8CF57F
:10476000002DE8D02DBAB5FA85F424F0070423FA19
:1047700004F122FA04F202F0FF0001F0FF01FDE86B
:104780000445A0EB010070474FEAC40420F0030089
:1047900050F8082B21F0030151F8083B0CFA04F4FF
:1047A00062EA040263EA0403C9E710F003041AD0C2
:1047B000A1EB040120F00300E40750F8042B06D01D
:1047C0000FD28B785FFAA2F4E41A06D12BB1CB7822
:1047D0005FFAB2F4E41A00D11BB920465DF8104B21
:1047E000704701F1040150F8042BCC0721F00301BC
:1047F00051F8043B48D824D222F07F4482FA4CF589
:1048000094EA1325A5FA8CF50AD165B951F8043B51
:1048100084EA0204B4EB036F0ED150F8042BEBE7EB
:104820004FEA132355E035F07F454DD10878FDE878
:104830000445C0F1000070474FEA126203F0FF0325
:1048400047E002EA1C4482FA4CF594EA1345A5FAC3
:104850008CF50AD165B951F8043B84EA0204B4EB43
:10486000034F0CD150F8042BEBE74FEA134330E031
:1048700015EA1C4528D10B884FEA124229E04FEA7D
:10488000124203EA1C4324E002F0FF0482FA4CF5D2
:1048900094EA1365A5FA8CF50AD165B951F8043B81
:1048A00084EA0204B4EB032F09D150F8042BEBE7A0
:1048B0004FEA13630DE015F0FF0F05D10B684FEAC7
:1048C000122223F07F4304E04FF00000FDE804458E
:1048D000704712BA1BBA82FA4CF482EA0304A4FAB3
:1048E0008CF5B5FA85F402FA04F203FA04F34FEA00
:1048F0001260FDE80445A0EB136070470000000063
:1049000090F800F06DE9024520F007016FF0000C0F
:1049100010F0070491F820F040F049804FF00004B7
:104920006FF00700D1E9002391F840F000F1080092
:1049300082FA4CF2A4FA8CF283FA4CF3A2FA8CF3CA
:104940004BBBD1E9022382FA4CF200F10800A4FA31
:104950008CF283FA4CF3A2FA8CF3E3B9D1E9042385
:1049600082FA4CF200F10800A4FA8CF283FA4CF3BC
:10497000A2FA8CF37BB9D1E9062301F1200182FA76
:104980004CF200F10800A4FA8CF283FA4CF3A2FA7C
:104990008CF3002BC6D0002A04BF04301A4612BA8A
:1049A000B2FA82F2FDE8024500EBD2007047D1E98D
:1049B000002304F00305C4F100004FEAC50514F01C
:1049C000040F91F840F00CFA05F562EA05021CBFED
:1049D00063EA050362464FF00004A9E72DE9F04FB2
:1049E000474C83460E46D4F800E000E026463446A5
:1049F00014F8015B0EEB0500407800F0080000F0B1
:104A0000FF080028F2D12D2D5CD02B2D04BF757826
:104A1000B41C002B3ED0102B60D09A46B8F1000F8A
:104A20000CBF6FF000404FF000400027B0FBFAF9D8
:104A3000BC460AFB19000CE0303DAB4219DD7E1C80
:104A400005D0CC4523D820D00AFB0C5C012714F8F4
:104A5000015B0EEB0506767816F0040FECD116F02C
:104A6000030606D0012E14BF57263726AD1BAB42D6
:104A7000E5DC7B1C16D0B8F1000F10D16046002A8F
:104A800039D0DFB91160BDE8F08F8542DCDD4FF031
:104A9000FF37DCE7302D1AD00A239A46BEE7CCF167
:104AA000000CEBE7B8F1000F4FF022030CBF6FF0E2
:104AB00000404FF00040CBF80030F2B1611E1160B1
:104AC000BDE8F08FB41C75784FF00108A1E723789A
:104AD00003F0DF03582B08D008239EE7302D9CD12C
:104AE000207800F0DF00582897D14FF0100A657841
:104AF0005346023492E7BDE8F08FBDE8F08F00BF67
:104B00008C02002010B4044C13460A46014620686B
:104B100010BCFFF763BF00BF2802002010B4044C94
:104B200013460A460146206810BCFBF755BB00BF80
:104B300028020020F8B50E461446054610B18369D8
:104B4000002B41D0254B9C4243D0254B9C4242D068
:104B5000244B9C4208BFEC68A389A269A2601A0793
:104B600021D52369FBB122686169D31A8B42F7B260
:104B700021DA0133A168501C0139A1602060167050
:104B800062699A4206D0A389DB0701D50A2F01D0BA
:104B90003846F8BD21462846FFF71EF80028F7D012
:104BA0004FF0FF37F4E72146284600F025F80028AB
:104BB000F6D12369D7E721462846FFF70DF80028EC
:104BC000EED122680123D5E7FFF740F9034B9C4261
:104BD000BBD16C68C0E7AC68BEE700BFD464000816
:104BE000B464000894640008024B0A460146186841
:104BF000FFF7A0BF28020020384B70B51D6806469D
:104C00000C4615B1AB69002B42D0354B9C4245D0C8
:104C1000344B9C4258D0344B9C4208BFEC68B4F9EA
:104C20000C2093B219070CD52069A8B113F001022A
:104C30001ED0636900225B42A361A260F0B1002034
:104C400070BDDD0642D558072AD4206942F008031A
:104C5000A3819BB20028E9D103F42072B2F5007F52
:104C6000E4D03046214600F06FF8A3892069DDE7E3
:104C7000990758BF6269A2600028E0D1B4F90C30EE
:104C80001A06DDD543F04003A3814FF0FF3070BD1D
:104C90002846FFF7DBF8124B9C42B9D16C68BEE79F
:104CA000616B51B104F14403994204D03046FFF7DF
:104CB000E3FAB4F90C2000236363002320696360E6
:104CC00022F024022060C1E7AC68A8E742F040026D
:104CD000092333604FF0FF30A28170BD280200200D
:104CE000D4640008B46400089464000870B50C46ED
:104CF000B1F90E10002990B015461E4613DB01AA2B
:104D0000FBF778FA00280EDB029A02F47042A2F553
:104D10000052B2FA82F252094FF4806300203260EE
:104D20002B6010B070BDA38900221B06326004D531
:104D3000402300202B6010B070BD4FF48063002032
:104D40002B6010B070BD00BF8A8992070B4606D554
:104D500001F1470201211A601A6159617047F0B5EB
:104D600083B001AB6A460C460546FFF7BFFF0099CA
:104D700006462846FFF7C6FAB4F90C30D0B1019ABE
:104D8000124F0099AF6243F08003A381206020613D
:104D900061611AB93343A38103B0F0BD2846B4F969
:104DA0000E10FBF72CFAB4F90C300028F2D043F0C7
:104DB0000103EFE79A05EFD404F1470243F0020341
:104DC0000121A381226022616161E5E7653C000861
:104DD0009368013B002B10B4936007DBCCB21368DF
:104DE000581C10601970204610BC70479469A3428B
:104DF00002DBCCB20A2CF2D110BCFFF79BBE00BF85
:104E000093B1F8B514460F460646D51801E0AC42FA
:104E100008D03A4614F8011B3046FFF7D9FF431C6F
:104E2000F5D1F8BD0020F8BD00207047936810B59B
:104E3000144613B95360184610BD00F0D1FB00238F
:104E4000A360636010BD00BF2DE9F04F9DB08846A0
:104E500014460393814618B18369002B00F00B813F
:104E60008B4B984500F00D818A4B984500F00C81E2
:104E7000894B984508BFD9F80C80B8F80C301D074D
:104E800040F1EF80D8F81030002B00F0EA8030239A
:104E90008DF82A302378814DDFF804A200212022EA
:104EA00009918DF82920002B00F08580252B2646BE
:104EB00003D117E0252B00F0868016F8013F002B68
:104EC000F8D1B6EB040B76D022465B464146484605
:104ED000FFF796FF01306ED0099B32785B4409934F
:104EE000002A68D000234FF0FF31721C049307930F
:104EF00006938DF853301A930591012604E0049926
:104F000006FA03F30B430493144664482178052200
:104F100000F0EEFC621C431B0028F0D1049BD80675
:104F200044BF20228DF853201907217844BF2B223B
:104F30008DF853202A2968D0A1F13002092A0BD814
:104F4000079B14F8011F03EB830302EB4303A1F15A
:104F50003002092AF5D907932E293FD00322504861
:104F600000F0C6FC48B10499CAEB0000402202FAE6
:104F700000F041EA000301340493217849488DF898
:104F800028100622013400F0B3FC00285FD0464B05
:104F9000EBB103AB00934246444B04A94846AFF340
:104FA000008007467A1C06D0099B3B44099323786E
:104FB000002B7FF47BAFB8F80C305B0658D409980F
:104FC0001DB0BDE8F08FB6EB040B8BD07CE7039BE4
:104FD000073323F0070308330393E5E761782A29B1
:104FE0001DD0A1F130020023092A04F10104059328
:104FF000B4D814F8011F03EB830302EB4303A1F1C0
:105000003002092AF5D90593A8E7039A11680432FA
:105010000029039215DB0791617801349CE7039B1B
:105020001A680592002A03F104030393B8BF4FF0F6
:10503000FF3204F10203AEBFA178A17805921C46AD
:105040008CE7494243F0020307910493E4E703AB82
:1050500000934246154B04A9484600F0CDF8074698
:10506000A0E741464846FFF7C7FD00283FF40FAFD1
:105070004FF0FF30A4E7FEF7E9FE054B98457FF4BB
:10508000F3AED9F80480F8E6D9F80880F5E600BF59
:10509000D4640008B4640008946400080066000842
:1050A000086600080C66000800000000014E0008B9
:1050B00010B4044C13460A460146206810BCFFF7A2
:1050C000C3BE00BF280200202DE9F0470C469146E0
:1050D0000969A268DDF820808A42B8BF0A46C9F88B
:1050E000002094F8431006461F4611B10132C9F85A
:1050F0000020236899065DD5D9F800200232C9F84E
:105100000020236813F0060F19461DD1E1688A1AA2
:10511000002AD8BF194617DD04F1190A002505E059
:10512000E368D9F800209B1AAB420CDD01235246FC
:1051300039463046C047013005F10105F0D14FF046
:10514000FF30BDE8F087216894F84330003318BF82
:1051500001238A060AD5E1185A1C302081F8430041
:10516000224494F8451082F84310023304F14302BC
:1051700039463046C0470130E1D0236803F00603CA
:10518000042B29D0A36822699342C8BF4FF00009BD
:105190002FDD9B1A99441A34002501E04D4528D093
:1051A0000123224639463046C047013005F101054A
:1051B000F4D1C4E713F0060F08D1E168D9F8002054
:1051C0008A1A002AD8BF1946A6DCBDE794F84330F6
:1051D000003318BF0123C9E7D9F80000E168A368CC
:1051E0002269091A934221EAE179D2DCB9F1000F70
:1051F000D1D10020BDE8F0872DE9F0430C46097EAF
:1052000085B06E29064617460C98984604F1430C63
:105210005AD01AD8632900F0128100F2D6800029F2
:105220005CD0582940F0F58084F845102268036866
:10523000DFF864E2150603F104011ED4550653BFDE
:105240001B6801601B88016019E0732900F0CF80A2
:105250007ED86F2900F0E480702940F0DA8022685F
:1052600042F020022260782384F845300368DFF89A
:105270002CE2150603F10401E0D51B680160D0079C
:1052800044BF42F020022260002B40F09080226850
:1052900022F0200222601021002284F8432060685E
:1052A000A0600028C0F28880226822F004022260F8
:1052B000002B62D1002840F08180654608296AD021
:1052C000C5EB0C0323610CE023681A0640F1D5807E
:1052D00003686269191D01601B681A600023654636
:1052E0002361CDF800803B4603AA21463046FFF7F4
:1052F000EBFE013021D02A46236939463046C047AB
:1053000001301AD02368039813F0020FE36819D014
:105310001A1A002A16DD04F11909002504E0E368D1
:1053200003981A1AAA420DDD01234A46394630462F
:10533000C047013005F10105F1D14FF0FF3005B054
:10534000BDE8F0839842B8BF184605B0BDE8F083C9
:10535000752965D078295CD1226884E76168A160ED
:105360002D200029C3F1000384F8430021DB22F043
:105370000402DFF824E122600A216546B3FBF1F262
:1053800001FB123013461EF8002005F8012D002BFA
:10539000F4D1082994D12368D90791D5626823698B
:1053A0009A428DDC302305F8013C013D88E710214D
:1053B00072E7DFF8E4E00A21002BDED19EF800302E
:1053C00084F8423004F1420578E7642901D0692964
:1053D0001FD122680368150603F104013AD51B6842
:1053E0000160002BBADBDFF8B0E00A2157E7036861
:1053F0006268191D01601D680021284600F078FAD6
:10540000002846D0401B60602061002384F84330B0
:1054100067E7012384F84210236104F14205F4E7B1
:1054200023681A061ED503681A1D1B680260227EB7
:10543000DFF864E06F2A14BF0A2108212CE7036813
:105440001A68191D0123016004F1420584F8422005
:105450002361DAE7550653BF1B680160B3F90030DA
:105460000160BEE713F0400F036803F1040215BFAB
:1054700002601B681B880260D9E713F0400F0368C5
:10548000626903F1040101601B6814BF1A801A608D
:1054900024E76068B8E700BF1466000828660008C3
:1054A000838903F00903092B01D000207047FEF720
:1054B000C5BB00BFF8B50C46054610B18369002B8B
:1054C00045D0424B9C4247D0414B9C426FD0414B10
:1054D0009C4208BFEC68B4F90C2093B200219F06EF
:1054E000616031D45E0722D5616B61B104F1440380
:1054F000994202D02846FEF7BFFE236C636000206D
:105500006063002B43D12369002B52D0B4F90C7097
:10551000BEB2B30722D12269226028466369656A58
:10552000216AA8470028606009DD0020F8BDD80680
:1055300044D519072ED442F00402A281E3E7A389DF
:105540001DD143F02003A3814FF0FF30F8BDFEF7DB
:105550007DFC1E4B9C42B7D16C68BCE71E4B1F49BB
:1055600018680123A38106F00906FEF78FFC092EB7
:10557000A781D0D121462846FEF796FACBE7002234
:1055800043F04003A38162604FF0FF30F8BDE36B4E
:105590002360F8BD21462846FEF71EFB0028D3D124
:1055A000B4F90C20A060A06122F00802C3E7AC6847
:1055B00091E721462846FFF7C7FBA7E742F04002E4
:1055C00009232B604FF0FF30A281F8BDD46400089E
:1055D000B464000894640008F4640008A15400084E
:1055E0009368002B76D02DE9F04F8B8985B00C465F
:1055F00019070190164629D522693AB303F002082B
:105600001FFA88F0356800282FD04FF00009B44FFA
:10561000C846B246B84543464A4628BF3B4601986D
:10562000B8F1000F50D0216AA66AB047002871DD9A
:10563000DAF808301B1A8144C0EB0808CAF80830B1
:10564000002BE7D1002005B0BDE8F08F214601987E
:10565000FFF7D2FA002840F03A81A389356803F0B9
:1056600002081FFA88F00028CFD113F001095BD19E
:105670004F4602961FB39A05D4F808802CD54745AB
:10568000C246C0F0A48013F4906F40F0B18020684F
:1056900052464946FEF73EFDA0682368C8EB00006D
:1056A0005344A06023603846029A93681B1A8144D1
:1056B0003F1A9360002BC5D0A389002FDBD1D5F80A
:1056C00000906F680835D5E7D5F80090D5F80480CC
:1056D00008359FE70020704720682369984203D867
:1056E00061698F4280F0B780B84528BFB84642460E
:1056F0004946FEF70FFDA3682268C8EB0303424446
:10570000A3602260002B49D121460198FEF764FA7C
:10571000002843D0B4F90C3043F040034FF0FF3081
:10572000A38105B0BDE8F08F804602908246814695
:10573000B9F1000F2AD0029B002B4CD020682369BE
:105740006269C845C34628BFCB4698425F4604D924
:10575000A36813449B4500F39080934520DB1346D8
:10576000A76A216A01985246B847071ED2DDB8EBF6
:10577000070823D0B368DB1BBA44C7EB0909B36041
:10578000002B3FF45FAFB9F1000FD4D10023D5F85F
:1057900000A0D5F8049002930835C9E7404683E796
:1057A0005A465146FEF7B6FCA2682368CBEB0202CC
:1057B0005B44B8EB0708A2602360DBD12146019867
:1057C000FEF70AFA0028A5D1CDF80880D2E72068B4
:1057D000B846BA465CE74A460A21504600F088F8C7
:1057E00000286FD001300123CAEB00080293A5E71F
:1057F00062692068216902EB4208C1EB000A08EBEC
:10580000D8780AF101004FEA68083844404542461A
:1058100084BF804642465B0542D511460198FEF79B
:1058200071FD8346002855D052462169FEF7D8FB0A
:10583000A38923F4906343F08003A381CAEB080398
:105840000BEB0A00C4F81480C4F810B02060A36009
:10585000B846BA461CE76FF00043BB4228BF3B4640
:105860004A4693FBF1F30198A66A01FB03F3216A10
:10587000B04700283FF718AF4CE71A46514603934C
:10588000FEF748FC2268039B01981A4422602146D7
:10589000FEF7A2F9039B00287FF43CAF1F4666E7A2
:1058A000019800F075F883460028C7D1019D216951
:1058B0002846FEF7E1FCB4F90C300C2223F08003FB
:1058C0002A6029E7012309F10108029336E74FF026
:1058D000FF30B8E6019A0C231360B4F90C301BE7D3
:1058E00000FCFF7F0000000000000000000000003E
:1058F00001F0FF01102A2BDB10F0070F08D010F881
:10590000013B013A8B422DD010F0070F42B3F6D184
:10591000F0B441EA012141EA014122F007047FF09D
:1059200000070023F0E80256083C85EA010586EAF4
:10593000010685FA47F5A3FA87F586FA47F6A5FA30
:1059400087F68EB9EED1F0BC01F0FF0102F007023C
:1059500032B110F8013B013A83EA010313B1F8D1E7
:105960000020704701387047002D06BF35460338C8
:10597000073815F0010F07D1013015F4807F02BF01
:10598000013015F4C03F0130F0BC0138704700BF52
:10599000F9B1F8B506461546B2B10C4600F01CF850
:1059A000854201D82046F8BD29463046FEF7AAFCBC
:1059B000074668B12A462146FEF712FB30462146CB
:1059C000FEF75AFC3846F8BDFEF756FC2846F8BDEF
:1059D000F8BD1146FEF796BC51F8040C0028BEBF76
:1059E000091851F8043CC018043870474E4D49203E
:1059F00048414E444C4552004D454D204D414E418D
:105A000047452048414E444C45520042555320469C
:105A100041554C542048414E444C45520055534149
:105A20004745204641554C542048414E444C455230
:105A3000004445425547204D4F4E2048414E444C6E
:105A400045520044554D4D592048414E444C455215
:105A5000000A49535220737461636B206F7665723C
:105A6000666C6F77656400537461636B20706F6957
:105A70006E74657220636F727275707465642C2029
:105A8000726573657420746F20746F70206F662068
:105A9000737461636B000A436F6E7465787420627F
:105AA00065666F726520686172646661756C743AD0
:105AB0000020202072303A2030782530386C780A67
:105AC00020202072313A2030782530386C780A2036
:105AD000202072323A2030782530386C780A202025
:105AE0002072333A2030782530386C780A00202034
:105AF0007231323A2030782530386C780A202020F4
:105B00006C723A2030782530386C780A202020706A
:105B1000633A2030782530386C780A202070737210
:105B20003A2030782530386C780A0A004653522FD4
:105B30004641523A0020434653523A2030782530AD
:105B4000386C780A0020484653523A203078253085
:105B5000386C780A0020444653523A203078253079
:105B6000386C780A0020414653523A20307825306C
:105B7000386C780A0020424641523A20307825306D
:105B8000386C780A004D4D4641523A203078253025
:105B9000386C780A004D697363004558435F52457D
:105BA000543A2030782530386C780A004174746596
:105BB0006D7074696E6720746F207265636F6E73A9
:105BC000747275637420737461746520666F7220DB
:105BD000646562756767696E672E2E2E00496E20B8
:105BE0004744423A0A2020736574202470633D3094
:105BF00078256C780A20206672616D6520300A2055
:105C00002062740A000A49535220737461636B2046
:105C10006F766572666C6F77656420627920617457
:105C2000206C656173742025642062797465732E1D
:105C30000A0048415244204641554C542048414EA8
:105C4000444C4552004641494C454420415353453C
:105C50005254494F4E2E0025700A002A2A2A2052FB
:105C6000494F54206B65726E656C2070616E69637C
:105C70003A0A25730A0A002A2A2A2068616C746588
:105C8000642E0A0A006D61696E28293A20546869F9
:105C9000732069732052494F54212028566572732E
:105CA000696F6E3A20554E4B4E4F574E2028627505
:105CB000696C646469723A202F686F6D652F656C3A
:105CC0006F7065732F50464531352F52494F542917
:105CD000290A0069646C65006D61696E005F51009E
:105CE000095E0008115E00081A5E0008235E0008C5
:105CF000295E0008315E00083A5E0008435E000835
:105D00004C5E0008545E00085C5E000873746174A9
:105D100065006E616D650009706964207C20252D29
:105D20003231737C20252D397351207C20707269AB
:105D3000207C20737461636B202028207573656458
:105D400029207C2062617365206164647220207C5C
:105D50002063757272656E7420202020200A00096D
:105D600020202D207C206973725F737461636B2027
:105D700020202020202020202020207C202D2020BA
:105D80002020202020202D207C2020202D207C2041
:105D9000253669202825356929207C202531307059
:105DA000207C20253130700A000925336869207C69
:105DB00020252D323073207C20252D387320252E70
:105DC0003173207C20253369207C202536692028EA
:105DD00025356929207C2025313070207C20253113
:105DE0003070200A007C0053554D00092535732082
:105DF000252D3231737C25313373253673202536BA
:105E0000692028253569290A0073746F70706564EC
:105E100000736C656570696E6700626C206D7574E7
:105E2000657800626C20727800626C2073656E6425
:105E300000626C207265706C7900626C20616E7912
:105E4000666C00626C20616C6C666C00626C206D2C
:105E5000626F780072756E6E696E670070656E6451
:105E6000696E670000440040000002000300024029
:105E7000020002400707002600480040000004001E
:105E8000090C0240080C024007070027070604021D
:105E9000010707050302000000300140070002402F
:105EA0000600024005000240040002400500000018
:105EB0000010000001000000003800400F04024004
:105EC0000E0402400D0402400C04024005000000D4
:105ED000004000000000000000000040FFFFFFFF46
:105EE00001000000001C0000000C0040FFFFFFFF4D
:105EF0000800000000320000020200000100000063
:105F000003000000060C02400A0C0240070C02408D
:105F1000040C0240756E6578706563746564206D6D
:105F2000657373616765207479706500676E72636D
:105F30005F6E65746465763A20706F737369626C26
:105F400079206C6F737420696E74657272757074E9
:105F50002E00556E6578706563746564206576659E
:105F60006E742072656365697665640041543836E5
:105F70005246327878206465766963652064726978
:105F8000766572207465737400496E697469616C1A
:105F9000697A696E672041543836524632787820E3
:105FA000726164696F206174205350495F25640AEF
:105FB00000726563765F7468726561640043726540
:105FC0006174696F6E206F662072656365697665BE
:105FD0007220746872656164206661696C65640032
:105FE000496E697469616C697A6174696F6E207356
:105FF00075636365737366756C202D2073746172AD
:1060000074696E6720746865207368656C6C206EB7
:106010006F77006966636F6E66696700436F6E66CF
:106020006967757265206E6574646576007478744E
:10603000736E640053656E642049454545203830D1
:10604000322E31352E34207061636B657400000090
:10605000136000081C600008351C00082D60000853
:1060600034600008411C000800000000000000002F
:1060700000000000496661636520253364202048E4
:1060800057616464723A20002C204C6F6E67204880
:1060900057616464723A20002C2050414E3A2030FF
:1060A0007825303478002865727229000A20202073
:1060B00020202020202020204164647265737320FA
:1060C0006C656E6774683A202575002C20536F75D7
:1060D0007263652061646472657373206C656E67BA
:1060E00074683A202575002C204D61782E50617916
:1060F0006C6F61643A202575000A20202020202042
:10610000202020202049507636204949443A20005A
:106110000A20202020202020202020204368616E9B
:106120006E656C3A202575002C2043682E706167DF
:10613000653A202575002C205458506F7765723AC7
:106140002025642064426D002C20776972656C659F
:106150007373002C20776972656400202020202052
:10616000202020200020205052454C4F4144002048
:10617000204155544F41434B0020205241570020AD
:10618000204155544F43434100202043534D41008B
:1061900075736167653A202573203C6966616365A4
:1061A0003E205B3C70616E3E5D203C616464723EEB
:1061B000203C746578743E0A00747874736E643A97
:1061C000202564206973206E6F7420616E20696ED3
:1061D000746572666163650A00747874736E643AFC
:1061E000204572726F72207072657065726172699B
:1061F0006E67206672616D6500747874736E643AC0
:10620000204572726F72206F6E2073656E64696EC6
:106210006700747874736E643A2073656E64202529
:106220007520627974657320746F200020285041B6
:106230004E3A2000556E6578706563746564204D34
:10624000485220666F7220696E636F6D696E6720B9
:106250007061636B657400424541434F4E00444199
:106260005441004D4143434D4400554E4B4E4F5712
:106270004E00446573742E2050414E3A20307825EC
:106280003034782C20446573742E20616464722E3F
:106290003A20000A5372632E2050414E3A20307843
:1062A000253034782C205372632E20616464722E62
:1062B0003A20000A53656375726974793A20003197
:1062C0002C2000302C20004672616D652070656EB8
:1062D000642E3A200041434B207265712E3A200013
:1062E00050414E20636F6D702E3A2000310056658C
:1062F0007273696F6E3A200025752C20005365710A
:106300002E3A2025750A007478743A20000A20205D
:1063100020202000525353493A2025752C204C51FF
:10632000493A2025750A0A0025303278000F0F0FF0
:106330000E0E0E0E0D0D0C0C0B0B0A0908070605B0
:10634000030003000300020002000100010000003E
:10635000FFFFFEFFFDFFFCFFFBFFF9FFF7FFF4FF70
:10636000EFFF0000152B00089D2A0008492A0008AD
:1063700095290008812B0008D92600080602020290
:106380000202020102030402020202020204FFFFEF
:106390003030303030303030007368656C6C3A200B
:1063A000696E636F72726563742071756F74696E64
:1063B000670068656C700044657363726970746926
:1063C0006F6E00436F6D6D616E6400252D3230730A
:1063D0002025730A002D2D2D2D2D2D2D2D2D2D2D0C
:1063E0002D2D2D2D2D2D2D2D2D2D2D2D2D2D2D2DDD
:1063F0002D2D2D2D2D2D2D2D2D2D2D2D0073686541
:106400006C6C3A20636F6D6D616E64206E6F7420EA
:10641000666F756E643A2025730A007265626F6F4D
:1064200074005265626F6F7420746865206E6F64CB
:1064300065007073005072696E747320696E666FC8
:10644000726D6174696F6E2061626F757420727510
:106450006E6E696E6720746872656164732E0000E9
:106460001B64000822640008113900083264000827
:10647000356400081B39000800000000000000001F
:10648000000000003031323334353637383941427C
:1064900043444546000000000000000000000000EA
:1064A00000000000000000000000000000000000EC
:1064B00000000000000000000000000000000000DC
:1064C00000000000000000000000000000000000CC
:1064D00000000000000000000000000000000000BC
:1064E00000000000000000000000000000000000AC
:1064F000000000002C0200204300000000202020AB
:106500002020202020202828282828202020202063
:106510002020202020202020202020202088101033
:10652000101010101010101010101010100404048F
:10653000040404040404041010101010101041414D
:10654000414141410101010101010101010101013B
:10655000010101010101010110101010101042424F
:10656000424242420202020202020202020202020B
:1065700002020202020202021010101020000000AB
:10658000000000000000000000000000000000000B
:1065900000000000000000000000000000000000FB
:1065A00000000000000000000000000000000000EB
:1065B00000000000000000000000000000000000DB
:1065C00000000000000000000000000000000000CB
:1065D00000000000000000000000000000000000BB
:1065E00000000000000000000000000000000000AB
:1065F000000000000000000000000000000000009B
:10660000232D302B20000000686C4C006566674528
:10661000464700003031323334353637383941425D
:1066200043444546000000003031323334353637BC
:0C66300038396162636465660000000098
:10663C0034120020000000006C0300204000000019
:10664C000000000000000000D35C0008D85C0008CB
:10665C0001010101010000002C02002000000000DB
:10666C00D4640008B46400089464000800000000BE
:10667C00000000000000000000000000F8640008AA
:10668C0000000000000000000000000000000000FE
:10669C0000000000000000000000000000000000EE
:1066AC0000000000000000000000000000000000DE
:1066BC00000000000000000000000000FC64000866
:0466CC002821000081
:0400000508000529C1
:00000001FF
